:1000000006308A00DC2E0000FF00030E8301A100F1
:100010000A08A0008A010408A2007708A300780853
:10002000A4007908A5007A08A600831383128C30F7
:100030008400001C1D280C1834288C308400801C7F
:1000400023288C183728220884002308F700240866
:10005000F8002508F9002608FA0020088A00210E79
:100060008300FF0E7F0E09008A110A124B288A11A5
:100070000A1285280A108A100A11820728340C34C3
:1000800001340634C822412A49274710C620492690
:100090005529C51000002B082D0203185C28A71253
:1000A00027088316870083128712271327088316D1
:1000B0008700831207136828A71227088316870072
:1000C00083128716271327088316870083120717C2
:1000D00003102C0D2D0203187428271227088316ED
:1000E0008700831207127A282712270883168700B1
:1000F000831207162D08C83C031C8028AD0A8128EE
:10010000AD010C108A110A122328D8012830D7001B
:10011000B20A3208183C0318B828B2010230570757
:100120008400831358188317800A00083B3C031887
:10013000B8280230570784008313581883178001AA
:10014000013057078400831358188317800A00086A
:100150003B3C0318B8280130570784008313581814
:100160008317800157088400831358188317800A67
:100170008C108A110A12232850294524C5205400C6
:10018000A519AE18E60843102000D327C12520107A
:1001900020100001A519AE18E6084310200006340F
:1001A0000934093406348034803480348034003497
:1001B000A71227088316870083128716271327089C
:1001C000831687008312071783168113091283127F
:1001D0009412A71227088316870083122716270870
:1001E000831687008312A711270883168700013022
:1001F000831294000030831694000108C739083830
:1002000081008530831290004830F8000638920053
:10021000F9308316920007309C00050885000330F2
:10022000F700F70B11291C0883120D1383169D018B
:10023000C03083128B0483168C140C141F149F106F
:100240001F159F111F1383121F179F1383169F17CC
:1002500083121F140030F8001F08C73978049F006C
:100260008A110A12F62E48308400831300080319FD
:1002700047290130F800F701F70B3C29F80B3B291F
:100280004A30F700F70B42294529800B392908002D
:100290000808F039D0004E080F39500488000715BF
:1002A00027112708831687000000831207112711E2
:1002B00027088316870083120800CC08031D6229D3
:1002C000871063298714A7102708831687008312D5
:1002D000CD0E4D08CE004821CD0E4D08CE00482150
:1002E0000D30F700F70B72290800C830C800332121
:1002F000F0308316880583128710A710270883160D
:10030000870083120711271127088316870083129D
:10031000B3013308023C031C95290230C800332185
:100320000330CE004821B30A89290D30F700F70BBE
:1003300097290230CE0048210D30F700F70B9E2997
:10034000B3013308023C031CB12933083A20B4003E
:10035000CC013408CD005D210230C8003321B30A3E
:10036000A1298A110A12032F831603178C170C1464
:100370000000000083128C080319DB290D08031309
:10038000B30003170F080313B40003170C0803137B
:10039000B5000130CC003508CD005D2133080317CE
:1003A0008D000313340803178F008D0A03198F0A79
:1003B0000313B429031703138A110A12112F83168A
:1003C0008C1002308312360784008313371883178A
:1003D00080013608840083133718831780010130A9
:1003E00036078400831337188317800183168C1413
:1003F0008312080001304802CA004908023C031D6C
:10040000032A4030CA074A088038CB00CC014B0889
:10041000CD005D21080047080C3A0319162A063A58
:1004200003191E2A073A0319242A292ACC0101306C
:10043000CD005D210230C8003321352A0130C800CB
:100440000230C900FA21352A0130C800C900FA215A
:10045000352A47081F3C031C2F2A0730C7050130E7
:10046000CC004708CD005D21352A0800831603170C
:100470008C170C140000000083120C087F3903193C
:100480007A2A0313B60003170D080313B7000317E6
:100490000F080313B8003608C7000B2237080317EC
:1004A0008D000313380803178F0083168C170C1464
:1004B0000000000083120C0D0E0D7F3903197A2AFB
:1004C0000313B60003170D080313B70003170F0833
:1004D0000313B8003608C7000B22370803178D0036
:1004E0000313380803178F008D0A03198F0A0313AB
:1004F000362A03170313080047080319EC2ACF0014
:100500004B080319EC2ACF0703188D2A7F30CF023E
:10051000031CEC2A0319EC2A912A8130CF07031817
:10052000EC2A4F08F700F801F901FA014808D30056
:10053000D3174908D2004A08D1001830CF00D001A3
:10054000511CBA2A4E08FA07031CAC2AF90A031DEB
:10055000AC2AF80A0319D0174D08F907031CB32A6F
:10056000F80A0319D0174C08C900C9174908F80739
:100570000318D017D00DF80CF90CFA0CD30CD20CD0
:10058000D10C0310CF0B9F2A0130F7070318EC2A78
:10059000F81BD12AD30DFA0DF90DF80DF703031945
:1005A000EC2AD31FE22AFA0A031DE22AF90A031DE4
:1005B000E22AF80A031DE22AF80CF90CFA0CF70AF1
:1005C0000319EC2A4808D0004C08D006D01FEA2AAC
:1005D000F817F02AF813F02AF701F801F901FA01E7
:1005E000080080308318CC06D101D2014808D00021
:1005F0004C08D00647080319E12BCF00F7004B0841
:100600000319EA2BCF020319862B031C442B4C0839
:10061000D500D5174D08D4004E08D300D2010310E1
:10062000D50CD40CD30CD20CCF0B0E2BD01F1B2B04
:100630005114FE2B51104F1051164A308400831371
:10064000132C5112D01B2E2B4F1C392BD50CD40C34
:10065000D30CD20CF70A0319F92B392BD51B3C2BE1
:100660000310D20DD30DD40DD50DF7030319F92BBB
:100670002E2B5117A62B51134808D000D01F422B08
:10068000D517F22BD513F22B4B08CF00F7004708F4
:10069000CF024808D500D5174908D4004A08D3002E
:1006A000D2010310D50CD40CD30CD20CCF0B502B91
:1006B000D01F5D2BD114FE2BD1104F10D1164E3010
:1006C00084008313132CD112D01B702B4F1C7B2B57
:1006D000D50CD40CD30CD20CF70A0319F92B7B2BB5
:1006E000D51B7E2B0310D20DD30DD40DD50DF703E2
:1006F0000319F92B702BD117A62BD1134C08D0005E
:10070000D01F842BD517F22BD513F22B4C08D50014
:10071000D5174D08D4004E08D300D01F932BD51306
:100720005115FE2B5111D2014F104A308400831312
:10073000132CD01BBC2B4808D0004F1CA62BD50C6B
:10074000D40CD30CD20CF70A0319F92BD21FB72BF8
:10075000D30A031DB72BD40A031DB72BD50A031DDB
:10076000B72BD50CD40CD30CF70A0319F92B511B5A
:100770003B2BD11B7D2BDB2B8030D506D51FC42B0B
:10078000FE2B4C08D000D12B4808D000D508031D03
:10079000D12BD408031DD12BD308031DD12BF70176
:1007A000F22BD51BDB2B0310D20DD30DD40DD50DA1
:1007B000F70BD12BF92BD01FDF2BD517F22BD5132D
:1007C000F22B4B08F7004C08D5004D08D4004E081A
:1007D000D300F22B4708F7004808D5004908D40099
:1007E0004A08D3005508F8005408F9005308FA00E5
:1007F000312CF701F801F901FA01312CD201D309AA
:10080000D409D509D209D20A031D0C2CD30A031D21
:100810000C2CD40A0319D50A51181A2BD1185C2BA9
:100820005119922BC12B0008D307031C1D2CD40A8D
:10083000031D1D2CD50A03194F1484030008D40787
:10084000031C252CD50A03194F1484030008801FAC
:10085000803AD50703184F14511A212BD11A632B54
:10086000992B0800C001BF01C10141081F3C031CB6
:100870004B2C1F151F193A2C83161E088312BF0715
:100880001E0803181E0FC0071030F700F70B462C88
:100890000000C10A352C400CFA003F0CF900FA0C9C
:1008A000F90CFA0CF90CFA0CF90CFA0CF90C0730EB
:1008B000FA057908F8007A08F9007908FA0078084A
:1008C000BF007A08C0008E30F7004008F8003F08EB
:1008D000F900FA01F808031D772C7908F800F901EE
:1008E0000830F702F808031D772CF7017F2C03105E
:1008F000F81B7E2CF90DF80DF703772CF8137030E8
:10090000CA009830C9002C30C8007E30C7007A0871
:10091000CE007908CD007808CC007708CB007C2287
:100920007708BF007808C0007908C1007A08C200C3
:10093000C4010408C3004410831B441483147A08C0
:10094000CA007908C9007808C8007708C700CD3008
:10095000CE002C30CD001330CC008730CB00F122FC
:100960004308840083134418831708004008C70015
:100970004408C706C71FC12C03110310C01B031472
:10098000F42C4008C7004308C8003F08C8020319F8
:10099000CF2CC71FF42C0308013A8300F42C440821
:1009A000C8004008C8020319DB2CC71FF42C030839
:1009B000013A8300F42C4508C8004108C802031915
:1009C000E72CC71FF42C0308013A8300F42C4608D7
:1009D000C8004208C8020319F32CC71FF42C0308EF
:1009E000013A8300F42C03100800F701F801F90123
:1009F000FA01CF01D001D101D2014E084D044C04BF
:100A00004B040319332D2030D3000310C70DC80D3C
:100A1000C90DCA0DCF0DD00DD10DD20D4E08520209
:100A2000031D1C2D4D085102031D1C2D4C085002A6
:100A3000031D1C2D4B084F02031C2D2D4B08CF020C
:100A40004C08031C4C0FD0024D08031C4D0FD10263
:100A50004E08031C4E0FD2020314F70DF80DF90DCA
:100A6000FA0DD30B052D4F308400831308000408C2
:100A7000BF003E08C1000319562D3D08CA003C08BE
:100A8000C9003B08C8003A08C700CE01CD0120309C
:100A9000CC008230CB007C227A08BD007908BC00F3
:100AA0007808BB007708BA00C10B3D2D3D08CA008D
:100AB0003C08C9003B08C8003A08C7004708B63CD4
:100AC000C700FA014808CB00C8170310C80CC90CAE
:100AD000CA0CFA0CF90CF80CF70CC70B652DCB1FE0
:100AE0007C2DF709F809F909FA09F70A0319F80A38
:100AF0000319F90A0319FA0A7A08BD007908BC003B
:100B00007808BB007708BA00BD1F932DBF03BF163E
:100B1000BA09BB09BC09BD09BA0A0319BB0A031902
:100B2000BC0A0319BD0A3B30C6009A30C500CA3062
:100B3000C400C3010A30C1003E080319BF0A3D08C2
:100B4000CA003C08C9003B08C8003A08C70046086C
:100B5000CE004508CD004408CC004308CB00F52466
:100B60000008BA00840A0008BB00840A0008BC0020
:100B7000840A0008BD00FD308407F708031DD32D4B
:100B80003E0A41020319D32D3F080319D52D0F3911
:100B900041020319CD2D0318052EBF1B052E3F1B47
:100BA000D52D2030012E2030BF05BF1EE32DBF12F2
:100BB0003E08031DBF037708BF002D30C7000B227E
:100BC0003F08F700BF013E084102031DF12D7708E1
:100BD000BF002E30C7000B223F08F7002030BF05B2
:100BE00000303030BF1E012EBF123E08031DBF0370
:100BF0007708BF002D30C7000B223F08F700BF0168
:100C00003030F7077708C7000B224608CA004508AE
:100C1000C9004408C8004308C700CE01CD01CC017B
:100C20000A30CB00F5247A08C6007908C500780898
:100C3000C4007708C300C10B9F2D0800831603175B
:100C40008C170C140000000003184D2E83120C08A2
:100C50007F390313BB0003170D080313BC000317F0
:100C60000F080313BD003B08C7000B223C08031705
:100C70008D0003133D0803178F0083168C170C1487
:100C80000000000083120313BA0B472E4A2E83166E
:100C900003174D2E6C2E8316031783120C0D0E0DA9
:100CA0007F390313BB0003170D080313BC000317A0
:100CB0000F080313BD003B08C7000B223C080317B5
:100CC0008D0003133D0803178F008D0A03198F0A47
:100CD00003100313BA0B1E2E08003908F80138025E
:100CE0000318752E3808F700812EF7010830BA0076
:100CF000B80DF70D390877020318F700F80DBA0B95
:100D0000782E080078083608B8006430B9006D26DF
:100D10007708B60078083030031D952EB71C9C2E3E
:100D2000B7199C2E371A2030982EB7113712371466
:100D3000F8077808C7000B223608B8000A30B90057
:100D40006D267708B60078083030031DAD2EB71930
:100D5000B12E371CB12E371A2030F8077808C7009B
:100D60000B223030B6073608C7000B220800F70107
:100D7000F801370803103818F707F70CF80CB81803
:100D8000F707F70CF80C3819F707F70CF80CB81937
:100D9000F707F70CF80C381AF707F70CF80CB81A25
:100DA000F707F70CF80C381BF707F70CF80CB81B13
:100DB000F707F70CF80C0800840183131F30830534
:100DC0008316861383128617AB01AC01B101B00103
:100DD000AF01AE01B20183161F149F141F159F119E
:100DE00007309C00FF308312A700D828A7122708DD
:100DF0008316870083128716271327088316870018
:100E0000831207177529CC014830CD005D210230CF
:100E1000C8003321CF3003178D0000308F0003133B
:100E2000B429CC010330CD005D210230C80033214C
:100E3000B7012830B600DF210230B3009630C80079
:100E40003321B30B1E2F8A1500288A111C2F630033
:10100000B7012830B6008A11DF218A150130C800E7
:101010000230C9008A11FA218A15BC3003178D00ED
:1010200000308F008A11031336228A15B901B801E6
:10103000B7017F30B600BA018A1132248A157708C9
:10104000BF007808C0007908C1007A08C200C40156
:101050000408C3004410831B441483147A08CA0094
:101060007908C9007808C8007708C7003108CE00A1
:101070003008CD002F08CC002E08CB008A11F122B9
:101080008A15430884008313441883177708BF0028
:101090007808C0007908C1007A08C200C6010408B7
:1010A000C5004610831B461483147A08CA007908C9
:1010B000C9007808C8007708C7003908CE0038088A
:1010C000CD003708CC003608CB008A11F1228A15F2
:1010D000450884008313461883177A08BE007908F0
:1010E000BD007808BC007708BB003E08C2003D0880
:1010F000C1003C08C0003B08BF00C601C501C401D7
:10110000C3018A11B6248A15031C8C2850303A0773
:10111000AB005A30AC008E28AB01AC018A113224EE
:101120008A157A08B1007908B0007808AF0077080E
:10113000AE000130C800C9008A11FA218A158A114F
:1011400032248A157708B6007808B7007908B80005
:101150007A08B900023084003908BD003808BC00A4
:101160003708BB003608BA000130BE008A113725A7
:101170008A15C23003178D0000308F00031404302D
:101180000313BA008A111E268A150930C8000130DF
:10119000C9008A11FA218A152808B6001130B70053
:1011A0008A1182268A153A30C7008A110B228A15C5
:1011B0002908B6000130B7008A1182268A153A3014
:1011C000C7008A110B228A152A08B6000130B70021
:1011D0008A1182268A150430B600FA30C8008A11B6
:1011E00033218A15B60BED282908033C0318092979
:1011F0000130C8000230C9008A11FA218A15423034
:1012000003178D0000308F008A11031336228A15D0
:1012100008298A1132248A157708B6007808B700A1
:101220007908B8007A08B900C2003808C100370848
:10123000C0003608BF00C601C5011630C4008630A4
:10124000C3008A11B6248A1503181628B70128305E
:10125000B6008A11DF218A150130B4003408B700C6
:101260003C30B8008A11B7268A1578086E3CB50064
:101270000130C8000230C9008A11FA218A15C53030
:1012800003178D0000308F008A11031336228A1550
:10129000B508031D4E29B4080319052AB901B80180
:1012A0001630B7008630B6008A1132248A157708C6
:1012B000BA007808BB007908BC007A08BD0039087C
:1012C000C2003808C1003708C0003608BF003D081A
:1012D000C6003C08C5003B08C4003A08C3008A1198
:1012E000B6248A15031C7729AB01AC017B29463053
:1012F000AB005030AC000130C800C9008A11FA219F
:101300008A158A1132248A157708B6007808B70042
:101310007908B8007A08B900023084003908BD00A5
:101320003808BC003708BB003608BA000130BE00E0
:101330008A1137258A15CC3003178D0000308F00B5
:10134000031404300313BA008A111E268A152A08D2
:10135000B5022908B7003C30B8008A11B7268A15B3
:1013600078086E3CF8002A087802B700B8003C30D4
:10137000B9008A116D268A157808B4002908B700CB
:101380003C30B8008A11B7268A1578086E3CF80000
:101390002A087802B6003408B7003C30B8008A1139
:1013A000B7268A1578083602B5000930C800013022
:1013B000C9008A11FA218A152808B6001130B70031
:1013C0008A1182268A153A30C7008A110B228A15A3
:1013D0003408B6000130B7008A1182268A153A30E7
:1013E000C7008A110B228A153508B6000130B700F4
:1013F0008A1182268A150430B600FA30C8008A1194
:1014000033218A15B60BFD2948298A110A12252F86
:02400E003A3F37
:00000001FF
